:100000002500A30404006100DF0C02000400DC0CE6
:10001000020004006600C90C0600040066070D0A11
:1000200066070D0A0607100A66070D0A0606140A77
:100030006B000400050C2D0066070D0A06071C0A5C
:10004000AB0266070D0A00000606200A04000B0238
:10005000B309A3046B00400E4306100AED021C0A0C
:100060006A0068000606AB020000B5090606AB028E
:1000700006064A0A2806590A00000606AB020A02CA
:1000800043074605430646040606AB022900080658
:10009000AB0A320A280500000606AB020A02430733
:1000A0004605430646040606AB0229000806AB0ACD
:1000B000320A280404000A024307460543064604A0
:1000C00029002607A6042606A60500000000000059
:1000D00000000000B5090B02B3092C000A02430717
:1000E00046054306460429006B00A30400000000F7
:1000F00000000000000000000000B509460786046B
:100100004606860500000000EC063F0A00000A02D1
:10011000430746054306460429000C023F0E2A0009
:10012000CC079F0A4604000000000000B509260520
:100130000000000000000000000000003F0A26044C
:1001400000000000B50900000000000000000000F1
:10015000000000003F0A4604B50926050000860499
:100160000000A6050D0AA30522006607080506067D
:10017000AB02E90043064604660708050606AB0223
:10018000E90043064604660708050606AB02E900D7
:1001900043064604660708050606AB02E900430667
:1001A0004604660708050606AB02E9004306460456
:1001B000660708050606AB02E90043064604660723
:1001C00008050606AB02E900430646046607080573
:1001D0000606AB02E9004306460466070805060664
:1001E000AB02E90043064604660708050606AB02B3
:1001F000E90043064604660708050606AB02E90067
:1002000043064604660708050606AB02E9004306F6
:100210004604660708050606AB02E90043064604E5
:10022000660708050606AB02E900430646046607B2
:1002300008050606AB02E900430646046607080502
:100240000606AB02E90043064604660708050606F3
:10025000AB02E90043064604660708050606AB0242
:10026000E90043064604660708050606AB02E900F6
:1002700043064604660708050606AB02E900430686
:100280004604660708050606AB02E9004306460475
:10029000660708050606AB02E90043064604660742
:1002A00008050606AB02E900430646046607080592
:1002B0000606AB02E9004306460466070805060683
:1002C000AB02E90043064604660708050606AB02D2
:1002D000E90043064604660708050606AB02E90086
:1002E00043064604660708050606AB02E900430616
:1002F0004604660708050606AB02E9004306460405
:10030000660708050606AB02E900430646046607D1
:1003100008050606AB02E900430646046607080521
:100320000606AB02E9004306460466070805060612
:10033000AB02E90043064604660708050606AB0261
:10034000E90043064604660708050606AB02E90015
:1003500043064604660708050606AB02E9004306A5
:100360004604660708050606AB02E9004306460494
:10037000660708050606AB02E90043064604660761
:1003800008050606AB02E9004306460466070805B1
:100390000606AB02E90043064604660708050606A2
:1003A000AB02E90043064604660708050606AB02F1
:1003B000E90043064604660708050606AB02E900A5
:0603C0004306460400089C
:100400002A082A082A082B083F083F083F083F0807
:100410003F083F083F083F083F083F083F083F08A4
:100420003F083F083F083F083F083F083F083F0894
:100430003F083F083F083F083F083F083F083F0884
:100440003F083F083F083F083F083F083F083F0874
:100450003F083F083F083F083F083F083F083F0864
:100460003F083F083F083F083F083F083F083F0854
:100470003F083F083F083F083F083F083F083F0844
:100480003F083F083F083F083F083F083F083F0834
:100490003F083F083F083F083F083F083F083F0824
:1004A0003F083F083F083F08800880088008800810
:1004B00080088008800880088008800880088008FC
:1004C000800880088008800880088008800840082C
:1004D00040084008400840084008400840084008DC
:1004E00040084008400840084008400840084008CC
:1004F00040084008400840084008400840084008BC
:1005000040084008400840084008400840084008AB
:10051000400840084008400840084008400840089B
:10052000400840084008400840084008400840088B
:10053000400840084008400840084008400840087B
:10054000400840084008400840084008400840086B
:10055000400840084008400840084008400800089B
:1005600000080008030805080608070809080A0823
:100570000A080B080C080D080E080E080F081008D2
:100580001008110812081208130813081408150897
:100590001508160816081708170818081808190863
:1005A000190819081A081A081B081B081C081C0837
:1005B0001C081D081D081E081E081E081F081F080D
:1005C00020082008200821082108210822082208E4
:1005D00022082308230823082408240824082508BF
:1005E000250825082608260826082708270827089A
:1005F00028082808280828082908290829082A0876
:021FFE00EE0FE4
:00000001FF
